BL51 BANKED LINKER/LOCATER V6.22                                                        09/28/2022  19:52:15  PAGE 1


BL51 BANKED LINKER/LOCATER V6.22, INVOKED BY:
C:\KEIL_V4\C51\BIN\BL51.EXE .\Release\system_FE81001.obj, .\Release\STARTUP.obj, .\Release\main.obj TO .\Release\Sample_
>> DrvMFA REGFILE (.\Release\Sample_DrvMFA.ORC) PRINT (.\Sample_DrvMFA.m51) RAMSIZE (256) CODE (0X0000-0X1FFF) XDATA (0X
>> 8000-0X87FF)


MEMORY MODEL: SMALL


INPUT MODULES INCLUDED:
  .\Release\system_FE81001.obj (SYSTEM_FE81001)
  .\Release\STARTUP.obj (?C_STARTUP)
  .\Release\main.obj (MAIN)
  C:\KEIL_V4\C51\LIB\C51S.LIB (?C_INIT)
  C:\KEIL_V4\C51\LIB\C51S.LIB (?C_IBP)


LINK MAP OF MODULE:  .\Release\Sample_DrvMFA (SYSTEM_FE81001)


            TYPE    BASE      LENGTH    RELOCATION   SEGMENT NAME
            -----------------------------------------------------

            * * * * * * *   D A T A   M E M O R Y   * * * * * * *
            REG     0000H     0008H     ABSOLUTE     "REG BANK 0"
            DATA    0008H     0004H     UNIT         ?DT?MAIN
            DATA    000CH     0002H     UNIT         ?DT?DELAY?MAIN
            DATA    000EH     0001H     UNIT         ?C?LIB_DATA
            IDATA   000FH     0001H     UNIT         ?STACK

            * * * * * * *  X D A T A   M E M O R Y  * * * * * * *
                    0000H     8000H                  *** GAP ***
            XDATA   8000H     0004H     ABSOLUTE     
* OVERLAP * XDATA   8000H     0004H     ABSOLUTE     
* OVERLAP * XDATA   8000H     0004H     ABSOLUTE     

            * * * * * * *   C O D E   M E M O R Y   * * * * * * *
            CODE    0000H     0003H     ABSOLUTE     
            CODE    0003H     012FH     UNIT         ?PR?MFAINIT?MAIN
            CODE    0132H     009DH     UNIT         ?C_C51STARTUP
            CODE    01CFH     0022H     UNIT         ?PR?MAIN?MAIN
            CODE    01F1H     001CH     UNIT         ?PR?DELAY?MAIN
            CODE    020DH     0007H     UNIT         ?C_INITSEG
            CODE    0214H     0001H     UNIT         ?PR?SYSTEMINIT?SYSTEM_FE81001



OVERLAY MAP OF MODULE:   .\Release\Sample_DrvMFA (SYSTEM_FE81001)


SEGMENT
  +--> CALLED SEGMENT
---------------------
?C_C51STARTUP
  +--> ?PR?MAIN?MAIN
  +--> ?C_INITSEG

?PR?MAIN?MAIN
BL51 BANKED LINKER/LOCATER V6.22                                                      09/28/2022  19:52:15  PAGE 2


  +--> ?PR?MFAINIT?MAIN

?PR?MFAINIT?MAIN
  +--> ?PR?DELAY?MAIN



SYMBOL TABLE OF MODULE:  .\Release\Sample_DrvMFA (SYSTEM_FE81001)

  VALUE           TYPE          NAME
  ----------------------------------

  -------         MODULE        SYSTEM_FE81001
  C:0000H         SYMBOL        _ICE_DUMMY_
  C:0214H         PUBLIC        SystemInit
  -------         PROC          SYSTEMINIT
  C:0214H         LINE#         38
  C:0214H         LINE#         39
  C:0214H         LINE#         41
  -------         ENDPROC       SYSTEMINIT
  -------         ENDMOD        SYSTEM_FE81001

  -------         MODULE        ?C_STARTUP
  C:0132H         SEGMENT       ?C_C51STARTUP
  I:000FH         SEGMENT       ?STACK
  C:0000H         PUBLIC        ?C_STARTUP
  D:00E0H         SYMBOL        ACC
  D:00F0H         SYMBOL        B
  D:0083H         SYMBOL        DPH
  D:0082H         SYMBOL        DPL
  N:0001H         SYMBOL        IBPSTACK
  N:0100H         SYMBOL        IBPSTACKTOP
  N:0080H         SYMBOL        IDATALEN
  C:0135H         SYMBOL        IDATALOOP
  N:0000H         SYMBOL        PBPSTACK
  N:0100H         SYMBOL        PBPSTACKTOP
  N:0000H         SYMBOL        PDATALEN
  N:0000H         SYMBOL        PDATASTART
  N:0000H         SYMBOL        PPAGE
  N:0000H         SYMBOL        PPAGEENABLE
  D:00A0H         SYMBOL        PPAGE_SFR
  D:0081H         SYMBOL        SP
  C:0132H         SYMBOL        STARTUP1
  N:0000H         SYMBOL        XBPSTACK
  N:0000H         SYMBOL        XBPSTACKTOP
  N:0800H         SYMBOL        XDATALEN
  C:0140H         SYMBOL        XDATALOOP
  N:8000H         SYMBOL        XDATASTART
  C:0000H         LINE#         126
  C:0132H         LINE#         133
  C:0134H         LINE#         134
  C:0135H         LINE#         135
  C:0136H         LINE#         136
  C:0138H         LINE#         140
  C:013BH         LINE#         141
  C:013DH         LINE#         145
  C:013FH         LINE#         147
BL51 BANKED LINKER/LOCATER V6.22                                                      09/28/2022  19:52:15  PAGE 3


  C:0140H         LINE#         148
  C:0141H         LINE#         149
  C:0142H         LINE#         150
  C:0144H         LINE#         151
  C:0146H         LINE#         170
  C:0149H         LINE#         185
  C:014CH         LINE#         196
  -------         ENDMOD        ?C_STARTUP

  -------         MODULE        MAIN
  C:0000H         SYMBOL        _ICE_DUMMY_
  D:0090H         PUBLIC        P1
  D:00B0H         PUBLIC        P3
  X:8000H         PUBLIC        mul_data_fp
  D:00A8H         PUBLIC        IE
  C:01F1H         PUBLIC        delay
  D:00B8H         PUBLIC        IP
  D:0008H         PUBLIC        aaa
  C:01CFH         PUBLIC        main
  X:8000H         PUBLIC        long_data
  D:0098H         PUBLIC        SCON
  D:0088H         PUBLIC        TCON
  X:8000H         PUBLIC        mul_data_char
  D:00C8H         PUBLIC        T2CON
  C:0003H         PUBLIC        MFAInit
  D:00D0H         PUBLIC        PSW
  -------         PROC          DELAY
  -------         DO            
  D:000CH         SYMBOL        i
  -------         ENDDO         
  C:01F1H         LINE#         39
  C:01F1H         LINE#         40
  C:01F1H         LINE#         43
  C:020CH         LINE#         44
  -------         ENDPROC       DELAY
  -------         PROC          MFAINIT
  C:0003H         LINE#         56
  C:0003H         LINE#         57
  C:0003H         LINE#         63
  C:0008H         LINE#         64
  C:000EH         LINE#         65
  C:0014H         LINE#         66
  C:001AH         LINE#         67
  C:0020H         LINE#         68
  C:0023H         LINE#         71
  C:002DH         LINE#         72
  C:0037H         LINE#         73
  C:0041H         LINE#         74
  C:004BH         LINE#         80
  C:0051H         LINE#         82
  C:0057H         LINE#         83
  C:005DH         LINE#         84
  C:0063H         LINE#         85
  C:0069H         LINE#         86
  C:006CH         LINE#         87
  C:0076H         LINE#         88
  C:0080H         LINE#         89
BL51 BANKED LINKER/LOCATER V6.22                                                      09/28/2022  19:52:15  PAGE 4


  C:008AH         LINE#         90
  C:0094H         LINE#         97
  C:0099H         LINE#         98
  C:009EH         LINE#         99
  C:00A3H         LINE#         100
  C:00A9H         LINE#         101
  C:00AFH         LINE#         102
  C:00B4H         LINE#         103
  C:00B9H         LINE#         104
  C:00BFH         LINE#         105
  C:00C5H         LINE#         107
  C:00C8H         LINE#         109
  C:00D2H         LINE#         110
  C:00DCH         LINE#         111
  C:00E6H         LINE#         112
  C:00F0H         LINE#         118
  C:00F5H         LINE#         119
  C:00FAH         LINE#         120
  C:0100H         LINE#         121
  C:0106H         LINE#         122
  C:0109H         LINE#         123
  C:0113H         LINE#         124
  C:011DH         LINE#         125
  C:0127H         LINE#         126
  C:0131H         LINE#         128
  -------         ENDPROC       MFAINIT
  -------         PROC          MAIN
  C:01CFH         LINE#         140
  C:01CFH         LINE#         141
  C:01CFH         LINE#         143
  C:01DAH         LINE#         146
  C:01E5H         LINE#         149
  C:01E8H         LINE#         152
  C:01EEH         LINE#         154
  C:01F0H         LINE#         155
  -------         ENDPROC       MAIN
  -------         ENDMOD        MAIN

  -------         MODULE        ?C_IBP
  D:000EH         PUBLIC        ?C_IBP
  -------         ENDMOD        ?C_IBP



FUNCTION REGISTER MASKS


FUNCTION . . . . . REG MASK
---------------------------

DELAY. . . . . . . @0xf000
MAIN . . . . . . . @0xf301
MFAINIT. . . . . . @0xf301
SYSTEMINIT . . . . @0x8000

*** WARNING L16: UNCALLED SEGMENT, IGNORED FOR OVERLAY PROCESS
    SEGMENT: ?PR?SYSTEMINIT?SYSTEM_FE81001
BL51 BANKED LINKER/LOCATER V6.22                                                      09/28/2022  19:52:15  PAGE 5



*** WARNING L6: XDATA SPACE MEMORY OVERLAP
    FROM:    8000H
    TO:      8003H

*** WARNING L6: XDATA SPACE MEMORY OVERLAP
    FROM:    8000H
    TO:      8003H

Program Size: data=16.0 xdata=12 code=533
LINK/LOCATE RUN COMPLETE.  3 WARNING(S),  0 ERROR(S)
